:06000000000080317B28A6
:100008007E1480312000921C76282100921C7628CC
:10001800200092108931BA2180312000EA006A0854
:100028006802031C7C146A08660203181D286A0803
:10003800E60021009D1825281C082000E900210061
:100048009D14CE0A0319CF0A0030200063026430E1
:100058000319620203183828E20A0319E30A62083E
:10006800643A63040319FC167C17033021004F021D
:10007800E83003194E02031C5328D00A0319D10A89
:10008800003051023D3003195002031C5028CC0A9D
:100098000319CD0AD001D101FC17CE01CF012000F0
:1000A8008C195A28E40A0319E50A75280F306502E5
:1000B800A13003196402031C6328FC15732803305C
:1000C8006502E93003196402031C6C287C15732847
:1000D800003065023330031964020318FC14E4018C
:1000E800E5017C162000911891107E1009008031DE
:1000F8007D286230FC01EB01840000308500093066
:100108008731F8278031CA308400003085002430D8
:100118008731F82780312030840001308500403055
:100128008731F8277E1020009431482C2100C00028
:100138005830AF00BC268031C3080319642D43082A
:10014800253A0319AF284008860001308700430884
:100158008100C00A9E28B501B601B301B4012B275E
:10016800803161268031031CEE282100B501B601DB
:100178000A302000A400A501210036082000A700AD
:10018800210035082000A6008C316D248031250817
:100198002100B600200024082100B5002B2780315B
:1001A800D03EDC00FF3003180030DD005C08210081
:1001B800B50720005D082100B63D2000D60A0319C6
:1001C800D70A560884005708850000086126803140
:1001D8000318BC28560884005708850000082E3AE2
:1001E800031D2E29210034172000D60A0319D70A27
:1001F8002100C101C2012B27803161268031031CF7
:10020800352956088400570885000008DC00DD0100
:10021800210042082000A500210041082000A40078
:100228000A30A600A7018C316D2480315C082407B0
:10023800DE005D08253DDF005E08D03E2100C100DC
:10024800FF3020005F3D2100C2002000D60A0319BC
:10025800D70AFF282100C101C201341635293415F7
:100268004429BC268031003A0319642D643A0319E5
:100278004429023A031933290F3A031944299E28BD
:1002880020000730DC01210034052000DD005C047B
:100298000319522C2100341E54290630C100C20112
:1002A8002F0886008701403FBD00413FBE00423F06
:1002B800BF000330AF073D08F1003E08F2003F08D9
:1002C800F300F401F501F6016A25803103187C2951
:1002D8003D08F1003E08F2003F08F3008D2680310A
:1002E8007108BD007208BE007308BF000330B30474
:1002F800BB01BC013F083E043D0403190C2ABD3074
:1003080048278031423FDE00433FDF000F30DF36B1
:10031800DE0CDD0CDC0C890B8B295D082100BC0090
:1003280020005C082100BB008230BC01BB07031C15
:10033800BC03FF30BB07031CBC0303302000A40030
:10034800A50121003C082000A70021003B0820004F
:10035800A6008C316D24803125082100BC002000C6
:1003680024082100BB000A30F700F8013C08FA0015
:100378003B08F9008C318224803178082100BC00C8
:100388007708BB00BC1FCC29FF30BB07031CBC038C
:100398003B03FF3A8B319E238031E72680310127CA
:1003A800210030082000AD00210031082000AE00F7
:1003B800210032082000AF008D31EE2580312A0857
:1003C8002100B00020002B082100B10020002C08DB
:1003D8002100B200392780318030F401F5003F3028
:1003E800F6006A2580310318FE29FF30BB07031C7D
:1003F800BC030C2A392780312030F401F500413044
:10040800F6006A258031031C0C2ABB0A0319BC0AB2
:100418004208FB268031031D142A0D3021004102B9
:1004280003183B2A210041088B31162380313908F3
:10043800C4003A08C5003B08C60021003D0820005A
:10044800C70021003E082000C80021003F08200006
:10045800C9008E318C26803144082100BD0020005F
:1004680045082100BE00200046082100BF002100E9
:100478003C08FB268031031D442A0A3021003B0238
:100488000318622A21003F083E043D0403199D2AEF
:100498003D080C278031CC258031440843044204B0
:1004A8004104031D9D2A21003C08FB268031031DC1
:1004B800602A023021003B02031C9D2A21003927B3
:1004C80080317030F4008930F5004030F6006A253C
:1004D80080310318712AF730722AF830BB07031CE1
:1004E800BC033B088B319E238031E7268031F10025
:1004F8003E08F2003F08F3003008F4003108F50028
:100508003208F6006127803174082100A6007308BC
:10051800A5007208A4007108A3002608BA002508DF
:10052800B9002408B8002308B700BD01BE01BF0107
:10053800D92A21003D080C278031CC258031CB26D3
:1005480080312100B7003A082000A30021003908B3
:100558002000A200210038082000A100210037084F
:100568002000A0006F2680312008D0002108D1008B
:100578002208D20021003D082000D30021003E08B7
:100588002000D40021003F082000D50095268031A6
:1005980050082100BD00200051082100BE002000A5
:1005A80052082100BF00BB01BC01C301C30AAC262D
:1005B800803117278031031DF12A200060082100AF
:1005C8003902031DF12A20005F0821003802031DAB
:1005D800F12A20005E0821003702031CF82AC30A0A
:1005E80043080A3A031DDB2A4308F42680314108F0
:1005F80020005C07DE002100420820005D3DDF008E
:1006080021003B0820005E07E00021003C08200094
:100618005F3DE10060082100B5022000610821006B
:10062800B63B4208410403191D2BFF30B507031CD4
:10063800B60333080339031D302B3608FB268031F7
:10064800031D292B013021003502031C352B210005
:10065800400857278031C00AFF30B507031CB6038E
:10066800212B21003308033903197B2B40085D2710
:100678008031792BAC268031F100013FF200D92678
:1006880080312126803174082100AA007308A9004E
:100698007208A8007108A7000A30322780312A089A
:1006A8002000AC00210029082000AB002100280808
:1006B8002000AA00210027082000A90096258031E3
:1006C80028082100AA00200027082100A9002000EE
:1006D80026082100A800200025082100A7004008BE
:1006E8008600013087002708303E8100C00AC30316
:1006F800430F3E2B3C08FB268031031D862B01301F
:1007080021003B02031C902B210040084027803128
:10071800BB07031CBC037E2B21004208FB2680314B
:10072800031D992B093021004102031C9E2B083020
:100738002100A02B21004108C300F4268031C1020A
:1007480020005D082100C23B43080319B22B400872
:100758008600013087002E308100C00A43088B31A3
:100768009E23803139082100A00020003A0821008A
:10077800A10020003B082100A20020082000AD00B5
:10078800210021082000AE00210022082000AF002F
:1007980021003D0801278D31EE2580312A08C1004E
:1007A8002B08C2002C08C300CC258031CB26803111
:1007B800422CAC268031F100013FF200D92680316D
:1007C8002126803174082100AE007308AD0072083C
:1007D800AC007108AB000A30322780312E082000A7
:1007E800AC0021002D082000AB0021002C082000BF
:1007F800AA0021002B082000A9009625803128088E
:100808002100AE00200027082100AD0020002608A6
:100818002100AC00200025082100AB00400886001C
:10082800013087002B08303E8100C00AAC26803199
:10083800A500013FA600023FA700033FA800210032
:100848003A082000AC00210039082000AB00210044
:1008580038082000AA00210037082000A9009625A2
:10086800803128082100BA00200027082100B9009B
:10087800200026082100B800200025082100B70024
:10088800C303430FDD2B4208410403199E28400887
:1008980040278031C107031CC203472C21002F08C1
:1008A800482780315C082100B70020005D0821003E
:1008B800B800890D893B8909B900BA00AF0AAF0AA7
:1008C800BA1F732C0330B304B709B809B909BA09B8
:1008D800B70A0319B80A0319B90A0319BA0A420868
:1008E8004104031D7F2C3A083904380437040319DE
:1008F800C10A0319C20AC301C30AAC2680311727EB
:100908008031031D972C2000600821003902031D47
:10091800972C20005F0821003802031D972C200027
:100928005E0821003702031C9E2CC30A43080A3ABA
:10093800031D812C4308212780314208803A20007A
:100948005E02031DAB2C2100410820005C02031845
:10095800B12C21004108C300C92C21004308F4260A
:1009680080314208803A2000DE005D08803A5E024D
:10097800031DC12C5C08210041020318C92C210069
:100988004308C100C201C11BC20321003608350457
:100998000319D62C330803390319D62CFF30B507B1
:1009A800031CB603341FF12C4208803A2000DC00F7
:1009B80021003608803A20005C02031DE62C210045
:1009C800350841020318EE2C21004108B5024208FF
:1009D800B63BF12C2100B501B6014308212780312F
:1009E8003608803A20005E02031DFE2C21003508DF
:1009F80020005C0203180A2D21004308F4268031E8
:100A0800B50220005D082100B63B0D2D2100B5017F
:100A1800B6013608350403191D2D400857278031C3
:100A2800FF30C00AB507031CB60336083504031D9A
:100A3800112D330803390319262D40085D2780310D
:100A48008100C00AFF30C107031CC203410A031911
:100A5800420A03199E280A3032278031420885004D
:100A6800410884008C308435850D8435850D8407D4
:100A78009A30853D003FF100013FF200023FF3004C
:100A8800033FF4003A08F8003908F7003808F60080
:100A98003708F500212680317408AC007308AB00D4
:100AA8007208AA007108A900962580312508303EF1
:100AB8002100C30040088600013087004308242D28
:100AC800400886000130870081010800F31F792D56
:100AD8007108003CF1007208031C720F003CF20020
:100AE8007308031C730F803CF300F61F882D7408ED
:100AF800003CF4007508031C750F003CF5007608EF
:100B0800031C760F803CF6008030F306F606760864
:100B18007302031D080075087202031D080074089B
:100B28007102080028082704260425040319C32D88
:100B3800F901F90AA81BA52DA535A60DA70DA80D25
:100B48009D2D28082C02031DB32D27082B02031DF9
:100B5800B32D26082A02031DB32D25082902031CDC
:100B6800BD2D2508A9022608AA3B2708AB3B280863
:100B7800AC3BA836A70CA60CA50CF90BA52D2C0888
:100B8800A8002B08A7002A08A6002908A500080025
:100B9800502780310310460D470DCD00CD08031DA9
:100BA800DA2DC101C201C301C401080050278031F8
:100BB8001730C736C60CC50C890BDD2D4508C80093
:100BC800C217C3014108C9004208CA004308CB0044
:100BD8008E30CC01CD02CD1FFD2D4D08803A8F3EC1
:100BE800031CD52DCC36CB0CCA0CC90CCD0FF62D59
:100BF8000A2E18304D020318D52DCD0803190A2ED8
:100C0800C935CA0DCB0DCC0DCD03012E48080319EB
:100C1800182EC909CA09CB09CC09C90A0319CA0A75
:100C28000319CB0A0319CC0A4C08C4004B08C300AB
:100C38004A08C2004908C10008002000A001A1011B
:100C4800A201A30174087304720471040319582ED5
:100C5800A401A40AF41B352EF135F20DF30DF40DA1
:100C68002D2EA035A10DA20DA30D74087802031D29
:100C7800472E73087702031D472E72087602031D5C
:100C8800472E71087502031C522E7108F50272086E
:100C9800F63B7308F73B7408F83B2014F436F30C62
:100CA800F20CF10CA40B352E2308F4002208F300F3
:100CB8002108F2002008F1000800F2003A30F101A2
:100CC800720203186D2E30307202031C6D2EF10172
:100CD800F10A710C08008E30F900FF302305031962
:100CE8007B2EA336A20CA10CA00CF90A712E2008A9
:100CF800F1002108F2002208F3007908F400F50158
:100D08008E3152267108A0007208A1007308A20053
:100D18000800730872047104031908008030F30690
:100D280008008030D2065308C4005408C50055088E
:100D3800C6005008C7005108C8005208C9008E31C3
:100D48008C264408D0004508D1004608D200080087
:100D580043082000DC008C30DD01DC35DD0DDC359E
:100D6800DD0D5C0784009A305D3D8500003F08007A
:100D780020005708DD005608DC00D60A0319D70AF8
:100D880084005D08850000082100C30008004408AD
:100D98002100BA00200043082100B90020004208C1
:100DA8002100B800200041080800023FF300033F7B
:100DB800F40021003A08F8003908F7003808F6006E
:100DC8003708F500080039082100B00020003A086B
:100DD8002100B10020003B082100B2003D080800B6
:100DE8002000DC00DD01DC1BDD0321000800803A67
:100DF8002000DC0080305C0208002000AA002100EE
:100E08003E082000AB0021003F082000AC0008008D
:100E18002000C10021003E082000C20021003F0838
:100E28002000C3000800DE00013FDF00023FE000B1
:100E3800033FE10021003A0208002000DC00DD0148
:100E4800DC1BDD035D08803ADE002100080020007D
:100E58005608840057088500000808002000A500EF
:100E6800A601A701A801210008003008F1003108F7
:100E7800F2003208F30008008600013087003030A5
:100E88008100FF30C00A080086008701403F20002B
:100E9800DC00413FDD0008004108C5004208C600EB
:100EA8004308C70008008600013087002030810011
:100EB80008008600013087002D347108F700720899
:100EC800F8007308F9000310780D790D2000A500CB
:100ED800A508031D742FF101F201F301F4010800C4
:100EE8007408F7007508F8007608F9000310780D03
:100EF800790DA400A40803196F2F7F30F217F301AE
:100F0800F517F601A001A101A201A301A5029830DD
:100F18002407F700A5021830A400A035A10DA20DE2
:100F2800A30D76087302031D9F2F75087202031D17
:100F38009F2F74087102031CA82F7408F10275080A
:100F4800F23B7608F33B2014F135F20DF30DA40BB8
:100F5800912FA51FBB2F2508803A973E031C6F2FA2
:100F6800A336A20CA10CA00CA50FB42FC82F1830C3
:100F7800250203186F2FA5080319C82FA035A10D46
:100F8800A20DA30DA503BF2F2308F4002208F30028
:100F98002108F2002008F1000800F800F4000030F1
:100FA8009531E4258731F73622000E150D13000020
:100FB80022008E100000FB0177087B020318E72F40
:100FC800FF30F900E82FF901FA0179089631072670
:100FD80087318030FB0A7B02031CE02F0D130000D1
:100FE800000022008E140800640080010131890B82
:040FF800F92F003499
:10129200F800F40000309531E4258931F736220058
:1012A2000E150D13000022008E100000FB017B08BA
:1012B200770603195E29F9016029FF30F900FA0166
:1012C20079089631072689318030FB0A7B02031C9C
:1012D20058290D130000000022008E1408000D137F
:1012E20021000D1322008D1221008D1223008D1278
:1012F20022000D1621000D1222000E1121000E11E6
:1013020023000E1122008E1421008E1023008E1055
:1013120022000D160D160D120D1200000000220003
:101322000D160D16F70100006430F70A7702031C50
:10133200942922000E110D13000022008E10F701D5
:101342007708823E84009A300318013E8500000827
:101352009631072689310A30F70A7702031CA12940
:101362000D130000000022008E140030F4019531AC
:10137200E42DF00122000C128E1221008E122200A6
:101382008C12132289310C160C12132289310C2271
:10139200893121008E1622000C2289310C228931DA
:1013A2000C160C120C160C120C1620008E1AF017CA
:1013B20022000C120C1620008E1A701722000C123A
:1013C2000C1620008E1AF01622000C120C162000A9
:1013D2008E1A701622000C120C1620008E1AF015AE
:1013E20022000C120C1620008E1A701522000C120C
:1013F2000C1620008E1AF01422000C120C1620007B
:101402008E1A701422000C120C128C168E122100ED
:101412008E12700808000C160C120C160C120C1608
:101422000C1208008E160C160C128E120C160C12D0
:101432000800713086008701403F2000A000413F34
:10144200A100423FA200433FA3000310220D230D3F
:10145200AD00AD08031D322AF101F201F301F401DE
:1014620008007430C2228A310310220D230DAC0011
:10147200AC0803192D2A7130860080304131413188
:1014820081047130413186007430CD228A31860068
:10149200803087014131413181047430413186000D
:1014A2007F30CD228A31A801A901AA01AB01AD0288
:1014B200A0302C07A000AD022030AC007430A8355B
:1014C200A90DAA0DAB0DC2228A3171308600403FB0
:1014D200A400413FA500423FA600433FA7002308C6
:1014E2002702031D7E2A22082602031D7E2A2108C6
:1014F2002502031D7E2A20082402031C922A74302E
:10150200C2228A31713086002008810241312108CD
:10151200813B41312208813B41312308813B7D31AE
:10152200281471308600870181354131810D4131A6
:10153200810D4131810DAC0B5F2AAD1FAC2A2D0804
:10154200803A9F3E031C2D2AAB36AA0CA90CA80C8C
:10155200AD0FA52AB92A20302D0203182D2AAD0875
:101562000319B92AA835A90DAA0DAB0DAD03B02AEE
:101572002B08F4002A08F3002908F2002808F100D9
:10158200080086008701403FA000413FA100423F82
:10159200A200433FA300080087014131413141319C
:1015A20081010800AE00E03EAF0022000E150D13CF
:1015B200000022008E1000002000B0012F08A400BD
:1015C2000630A501A600A7016D240030AA009830BC
:1015D200AB0024082A07AC0025082B3DAD003008DB
:1015E2002C0784002D0803182D0A85000008963167
:1015F20007268A3120000630B00A3002031CDF2A97
:1016020022000D130000000022008E14063021007B
:10161200DD0780305D02031C08008030DD070830E2
:10162200DE0A5E020318DE0108002000C3006E30ED
:101632004302031C612B0A30F6006430F1004308B8
:1016420014258A31FC248A31A3278A316D248A31F8
:1016520070278A314E278A316430F6004308FC2411
:101662008A31A3278A316D248A3194278A316027EF
:101672008A31EE258A31E3278A310A30F1004308A4
:1016820014258A31A3278A316D248A3125084027FF
:101692008A31CF278A31EE258A312A08BD002B08EC
:1016A200BE002C08BF003F30AA01AB01AC003D08D0
:1016B200AD003E08AE003F08AF00EE258A31B02FE4
:1016C2000B304302031C8B2B0A30F1004308142514
:1016D2008A31A3278A316D248A31250840278A312D
:1016E2000A30F6004308FC248A31A3278A316D248C
:1016F2008A3170278A3160278A31EE258A31E327C1
:101702008A313F30AA01AB01AC00CF278A31EE25E6
:101712008A31B02F3F30AA01AB01AC004308A327A6
:101722008A316D248A3156278A31AD00013FAE00DD
:10173200023FAF00EE258A31B02F2000C000C01F4B
:10174200042CC009C00A4008803A123E031CDB2B5D
:101752000A30B7278A31C3248A31F6278A31822494
:101762008A3168278A316D248A3170278A314E275F
:101772008A316430C9278A31F91BFA0382248A31FB
:1017820068278A316D248A3194278A3160278A3109
:10179200EE258A3185278A31C3248A319B278A31F3
:1017A2006D248A31250840278A31D6278A31EE25D1
:1017B2008A317E2FFB278A31031CFD2BF300A927D8
:1017C2008A31C3248A319B278A316D248A312508C4
:1017D20040278A310A30C9278A31F91BFA03822449
:1017E2008A3168278A316D248A3170278A316027CD
:1017F2008A31EE258A317E2FA3278A316D248A31E0
:1018020056278A31DD2F4008803A123E031C412CB4
:101812000A30B7278A31C3248A31F6278A318224D3
:101822008A3168278A316D248A31C2278A314E274C
:101832008A316430C9278A31F91BFA0382248A313A
:1018420068278A316D248A3125088500240884009E
:10185200913084079A3060278A31EE258A318527B4
:101862008A31C3248A319B278A316D248A317727B2
:101872008A314E278A31D6278A31EE258A317E2F48
:10188200FB278A31031C642CF300A9278A31C32465
:101892008A319B278A316D248A3177278A314E27F4
:1018A2008A310A30C9278A31F91BFA0382248A3124
:1018B20068278A316D248A31C2278A3160278A31AA
:1018C200EE258A317E2FA3278A316D248A3177272C
:1018D2008A31853D003FDD2FA801A901241C752C0A
:1018E2002608A8072708A93DA635A70DA536A40CEA
:1018F20025082404031D6F2C2908A5002808A4002C
:1019020008002000A101F81F8D2CF709F809F70A39
:101912000319F80AA101A10AFA1F962CF909FA097A
:10192200F90A0319FA0A0130A106A201A3017808F3
:1019320077040319B62CA001A00AF81BA32CF735D3
:10194200F80D9D2CA235A30D78087A02031DAB2C4D
:1019520077087902031CB22C7708F9027808FA3B5F
:101962002214F836F70CA00BA32C21080319BE2C65
:10197200A209A309A20A0319A30A2308F80022084C
:10198200F7000800F601F41FCD2CF309F409F30A5D
:101992000319F40AF601F60AF21FD42CF109F2092E
:1019A200F10A0319F20A720871040319EF2CF50106
:1019B200F50AF21BDF2CF135F20DD92C72087402F4
:1019C200031DE52C71087302031CEB2C7108F30252
:1019D2007208F43BF236F10CF50BDF2C7608031992
:1019E200F72CF309F409F30A0319F40A7408F20054
:1019F2007308F1000800F700F90176080319122DA7
:101A0200F801F80AF61B072DF635022DF93576088E
:101A12007702031C0F2D7608F7027914F636F80BBD
:101A2200072D79080800F3000830F400F501730867
:101A3200F2000730F236890B1B2D75357204F50062
:101A4200F33571087502031C282D7108F502F40B99
:101A5200182D750808002000D3000930F60076081A
:101A6200F500F517973186278A317508CE258A3118
:101A7200210000308E16CE258A310030CE258A31E3
:101A8200F7000C128C168E1221008E12770820009D
:101A9200D400D501D601D7015608F0270A30D40167
:101AA200F6007608F500F517973186278A31750812
:101AB200CE258A31210000308E16CE258A310030A3
:101AC200CE258A31F7000C128C168E1221008E124E
:101AD20077082000D40701300318D5070318D6076A
:101AE2000318D7075608F0270B30D401F600760802
:101AF200F500F517973186278A317508CE258A3188
:101B0200210000308E16CE258A310030CE258A3152
:101B1200F7000C128C168E1221008E12770820000C
:101B2200D40701300318D5070318D6070318D707BF
:101B3200CD30C4004C30C5003E30C6008030AA0112
:101B4200AB003930AC005708A3005608A200550874
:101B5200A1005408A00086316F268A312008AD000A
:101B62002108AE002208AF00EE258A312A08C700FC
:101B72002B08C8002C08C9008C264408D000450850
:101B8200D1004608D2005308860087015008C03FA2
:101B92005108C13F5208C23F0800F1008030F201F3
:101BA200F300F401F11FD82D22008E16DA2D220047
:101BB2008E12000022000C160000200073088E1AFC
:101BC200F204000022000C120830F135F336F40A58
:101BD2007402031CD32D720808002A08B0002B08D7
:101BE200B1002C08B2000310310D320DB300B3085E
:101BF200031DFF2DAA01AB01AC0108002D08B000A6
:101C02002E08B1002F08B2000310310D320DB800BA
:101C1200B808031D102EAA01AB01AC010800380858
:101C22007B3EB3072C08B8002F08B8068030B805F1
:101C3200FF30AB17AE17AD05AE050730AF01B401EB
:101C4200B501B601B7002A1C292E2D08EA278A31D0
:101C5200AC36AB0CAA0CAD35AE0DAF0DB70B242EC6
:101C62000930B7002A1C382E2D08EA278A31AC36F3
:101C7200AB0CAA0CB636B50CB40CB70B332E340829
:101C8200F1003508F2003608F3003308F400380892
:101C9200F50052267108AA007208AB007308AC0066
:101CA2000800740803195A2E730872047104031D84
:101CB200622EF101F201F3010800F40AF336F20C8C
:101CC200F10CFE3073050319702E5E2EF40AF10A30
:101CD2000319F20A0319F30AF336F20CF10CFF307E
:101CE20073050319792E672EF403F135F20DF30D06
:101CF200F21F752E741CF213F4367408F800F70103
:101D0200F6017608F1047708F2047808F3047508FE
:101D1200031DF31708004408CA004508CB00460813
:101D2200CC0003104B0D4C0DCF004708CA004808E9
:101D3200CB004908CC0003104B0D4C0DCE004F08D0
:101D42000319AF2E4E084F024E080318B72ECA00D1
:101D52004F08CA0219304A02031CB62E4708C400B3
:101D62004808C5004908C60008004E0803190800C3
:101D72004F084E020318C52E4F08CA004E08CA0269
:101D820019304A02031808000630CD00C61BCD17D1
:101D9200C91B4D17C517C601C817C9014E084F0206
:101DA2000318EA2EC735C80DC90DCE034E084F06DB
:101DB2000319E52ECD034D0807390319E52ED32E5D
:101DC200C636C50CC40CCF0A4F084E060319042FA1
:101DD200E12E4F084E020318042FC435C50DC60D5F
:101DE200CF034E084F060319002FCD034D080739C4
:101DF2000319002FEE2EC936C80CC70CCE0A4F08A5
:101E02004E06031DFC2ECD1F0F2FFF30C406C50644
:101E1200C606C40A0319C50A0319C60A4D1F1A2F9A
:101E2200FF30C706C806C906C70A0319C80A03193C
:101E3200C90ACD014408C7074508C83D4608C93D3F
:101E4200C91F2E2FFF30C706C806C906C70A0319C5
:101E5200C80A0319C90ACD01CD0A4708F10048088A
:101E6200F2004908F3004F08F4004D08F50052262D
:101E72007108C4007208C5007308C6000800850016
:101E820024088400343084079A30853D003FAA003C
:101E9200013FAB00023FAC000800853D003FAA00B5
:101EA200013FAB00023FAC00080025088500240872
:101EB2008400343084079A30853D003F0800853D18
:101EC200003FAD00013FAE00023FAF0008007808BE
:101ED200A5007708A4000330A600A7010800250882
:101EE2008500240884004F3084079A342508850031
:101EF200240884005B3084079A342A08B9002B082E
:101F0200BA002C08BB0008002A08BD002B08BE003E
:101F12002C08BF004008F300F401F31BF4030A305D
:101F2200F100F201080025088500240884006A30C7
:101F320084079A347208A5007108A4000330A60031
:101F4200A7010800A4000330A501A600A70108000C
:101F5200F401F31BF4030A30F100F20108002A082D
:101F6200B9002B08BA002C08BB000800F700F801E2
:101F72004008F300F401F31BF4036430F100F201B2
:101F820008002508850024088400763084079A34E6
:101F9200F700F8014008F900FA0108004008AD0016
:101FA2004108AE004208AF0008003D08AD003E08FF
:101FB200AE003F08AF000800B900013FBA00023F7F
:101FC200BB0008002A08C0002B08C1002C08C20070
:101FD2000800B4072E08B53D2F08B63D0800D7000B
:101FE2005508D6005408D50008007208FA00710896
:0E1FF200F90008004008803A753E40080800DB
:10289000FC107C11FC115B269431632694318C264C
:1028A00094318D1325008D172100C90122008D134D
:1028B0006430F100F2019425943122008D17C83064
:1028C000F100F2019425943121000530C90A490232
:1028D000031C562C20000C1C6F2C6B10702C6B14DE
:1028E0000A30F300F430F401F5000130F600A925B8
:1028F0008931702194319030F1000130F20094253B
:10290000943138269431B72794310030F401F40A19
:10291000E4259431C3302000B1009A30B200232660
:102920009431E327943194259431382694319127BA
:102930009431F426E9308D312C2594312100690839
:10294000C4006A08C5006B08C600E8302000BC2738
:1029500080319A209431ED279431D8259431E327A2
:102960009431942594318B172000E7012000670BE8
:10297000072D21004708200069060319072D690863
:102980002100C70044082000C400210045082000A1
:10299000C500210046082000C6004330AA00A1302F
:1029A000AB003D30AC007F30F900FA016908F90254
:1029B000031CFA03D8267908AD007A08AE007B081C
:1029C000AF008D31EE2594312A08C7002B08C800CE
:1029D0002C08C9008E318C26943144082100E9006E
:1029E000200045082100EA00200046082100EB00F5
:1029F000E9300B27943120006B18072DE830BC27F5
:102A000080319A209431ED279431D8259431E7080C
:102A1000031D0C2D6908E8006A082100C8007C1C11
:102A2000142D22008D137C1020006B183A2DF730E6
:102A3000D6009A30D700210048082000D800D901DC
:102A40006608DA002030DB0180319A2094312000C2
:102A50000030B301B30AD82521004808F70002303E
:102A60008731D127943120006808F700033089317D
:102A70004921943122008D1B632D2000E201E301E6
:102A80000030630232300319620203185D2D220008
:102A90000E130E160A30F100F201C7259431220000
:102AA0000E170E120A30F100F201C7259431E70823
:102AB000031D402D6908E800402D6A086802031CC8
:102AC000472D22008D17FC1C742DFC102000E60100
:102AD000E7016B18702D0730F700F8019927943142
:102AE000D7279431A92594317C1D902D7C1120008D
:102AF00069082100C70001302000E7006B188C2D09
:102B00000730F4000030E4259431D6302000B100C5
:102B10009A30B20023269431D7279431A9259431D5
:102B2000FC1DB62CFC11B62C7208710403190800A8
:102B3000F30128009C0120001211121D9D2D0A3066
:102B4000F30A7302031C992D0130F1020030F23BAD
:102B5000942DF436F30C0130F5020030F63B750A83
:102B60000319760A0319C32D22000E130E16E82747
:102B70009431C725943122000E170E12E8279431A4
:102B8000C7259431AB2D22000E130E120800200031
:102B90001211720871040319080028009C0120001A
:102BA000121DCF2D12110130F1020030F23BC92D60
:102BB000FB003308F4007B08E4259431203020002A
:102BC000B1000130B200232EF60022000E110D13C9
:102BD000000022008E1074080739B038072694319F
:102BE0007608023E890E0F391038072694310230DC
:102BF0007607F5000F3907260D13000000002200AC
:102C00008E1476082100DD007408DE000800F20052
:102C1000F3017208F100730A0E2EF135890B0D2EA7
:102C2000F11F152E22008D16172E22008D12000086
:102C300022000D17000022000D130830F30A730262
:102C400003180800092E31088400320885000008A6
:102C50000038031908003108840032088500000894
:102C60008A31D32294312000B10A0319B20A232EEB
:102C7000F8017808F4000030E425943122000E15A4
:102C80000D13000022008E100000F701003007260F
:102C900094318130F70A7702031C462E0D13000091
:102CA000000022008E140830F80A7802031C392E26
:102CB0000030F401E42DF030210099001A1F5E2E3F
:102CC0001A180800602E95120B1195111515951004
:102CD00015108B1235302000980021001110F930AA
:102CE00020009B003C309C0021009110F93028000E
:102CF0009600200092100E302800970021009214B8
:102D00000B17633028009D00200012110D302800A1
:102D10009E00210012110800951324008C018D01E2
:102D20008E0121000E1423000E1022000C10210031
:102D30000C1023000C1022008C1621008C1226008F
:102D40008C1222000C1221000C1226000C12220000
:102D50008E1221008E1226008E1223000C122200E9
:102D60000E1321000E1322000E1221000E1223005A
:102D70000E133D00A601A40122008D1721008D1322
:102D80003D009F0121008E1523008E1521000C149B
:102D900023000C1024000C141D3021009D0028304D
:102DA0009E009F0123008E1521008E159D140800A2
:102DB000A001FA1FE22EF909FA09F90A0319FA0A21
:102DC000A001A00A7908F1007A08F2008E30F30120
:102DD000F4002008F5008E3152267108F9007208BF
:102DE000FA007308FB0008000430F70014305B277A
:102DF0009431B430F7009A30F8000F30F900003009
:102E0000632794319530F70019305B2794310530F2
:102E1000F70014305B2F2000D3000430F70014308B
:102E20005B2720008030AA01AB004530AC00CD30DC
:102E3000C4004C30C500BE30C60053088600870170
:102E4000403FC700413FC800423FC9008E318C2639
:102E500094314408AD004508AE004608AF008D31FE
:102E6000EE2594312A08D0002B08D1002C08D2007E
:102E70005008C1005108C2005208C3008531CC255A
:102E800094314408D7004308D6004208D5004108D1
:102E9000D400F7000B305B279431CC2794310A30F3
:102EA0005B279431CC27943109305B27943105306E
:102EB000F70014305B2FF8007708F50078087D27BD
:102EC00094310C12DE2FFA00770884007808850010
:102ED0000008F5007A087D279431792FF70A031945
:102EE000F80A770884007808850000088D31CE251F
:102EF0009431F90B6E2F0C12DE2FF600F613862795
:102F000076088D31CE2575088D31CE2D22000C121C
:102F10008E1221008E1222008C1200000000000090
:102F200008000E1423000E1021000C1523000C11B4
:102F300008007708F4000030E425943122000E15D3
:102F40000D13000022008E100000F901003007264A
:102F500094318030F90A7902031CA62F0D1300006A
:102F6000000022008E147708F4000030E42DC030F9
:102F7000F1279431A030F12FD6009A30D7002100EC
:102F800069082000D80021006A082000D90021002B
:102F90006B082000DA00203420005508D4005608C1
:102FA000D5005708D600D7015408F70008001430A0
:102FB000F3006430F401F500F60108008C168E125F
:102FC00021008E120800E830F1000330F200080002
:102FD0007408F2007308F100080005302000B30007
:102FE0000034F40022000E110D13000022008E1098
:102FF000740807260D130000000022008E1408003C
:103000000034003400340034003400340034003420
:1030100000342F34003400340034003407340034DA
:1030200007340034003414347F3414347F341434BF
:10303000003424342A347F342A3412340034623485
:10304000643408341334233400343634493455346A
:103050002234503400340034053403340034003456
:10306000003400341C342234413400340034003441
:10307000413422341C3400340034143408343E34D7
:10308000083414340034083408343E340834083426
:10309000003400340034A034603400340034083488
:1030A00008340834083408340034003460346034A0
:1030B0000034003400342034103408340434023432
:1030C00000343E345134493445343E340034003405
:1030D00042347F344034003400344234613451345B
:1030E0004934463400342134413445344B3431348E
:1030F00000341834143412347F341034003427343C
:10310000453445344534393400343C344A34493448
:103110004934303400340134713409340534033413
:1031200000343634493449344934363400340634B2
:103130004934493429341E340034003436343634AA
:103140000034003400340034563436340034003453
:10315000003408341434223441340034003414343C
:10316000143414341434143400340034413422340C
:103170001434083400340234013451340934063430
:10318000003432344934593451343E3400347C34C0
:103190001234113412347C3400347F3449344934CD
:1031A0004934363400343E344134413441342234DD
:1031B00000347F344134413422341C3400347F34B1
:1031C000493449344934413400347F3409340934B2
:1031D0000934013400343E344134493449347A34BA
:1031E00000347F340834083408347F340034003429
:1031F00041347F344134003400342034403441348D
:103200003F34013400347F340834143422344134E0
:1032100000347F34403440344034403400347F3410
:1032200002340C3402347F3400347F3404340834E4
:1032300010347F3400343E344134413441343E3420
:1032400000347F34093409340934063400343E3400
:103250004134513421345E3400347F34093419341C
:1032600029344634003446344934493449343134FD
:103270000034013401347F340134013400343F34EC
:103280004034403440343F3400341F342034403420
:1032900020341F3400343F344034383440343F3419
:1032A0000034633414340834143463340034073481
:1032B00008347034083407340034613451344934EC
:1032C00045344334003400347F34413441340034D5
:1032D000003455342A3455342A34553400340034FB
:1032E000413441347F340034003404340234013436
:1032F00002340434003440344034403440344034E8
:1033000000340034013402340434003400342034F6
:10331000543454345434783400347F34483444348E
:10332000443438340034383444344434443420345D
:10333000003438344434443448347F34003438342E
:103340005434543454341834003408347E3409343A
:103350000134023400341834A434A434A4347C344A
:1033600000347F34083404340434783400340034B6
:1033700044347D3440340034003440348034843468
:103380007D34003400347F34103428344434003425
:103390000034003441347F344034003400347C3411
:1033A000043418340434783400347C34083404345D
:1033B00004347834003438344434443444343834B5
:1033C0000034FC34243424342434183400341834C5
:1033D000243424341834FC3400347C340834043469
:1033E00004340834003448345434543454342034CD
:1033F000003404343F3444344034203400343C340A
:103400004034403420347C3400341C342034403484
:1034100020341C3400343C344034303440343C34A8
:1034200000344434283410342834443400341C34F8
:10343000A034A034A0347C34003444346434543494
:103440004C344434143414341434143414341434D4
:10345000FF34FF34FF34FF34FF34FF34FF34813452
:10346000813481348134FF34003480343F34CD34AE
:10347000CC343D34D73423343C34123483343A349E
:10348000B734D1343834C6342734373438348634FA
:103490003534C034D6343334CC342B3432347034F5
:1034A00089343034E734DB342E34E5343C341E3494
:1034B0004234A2340D34003480343F34003420349C
:1034C00041340034C834423400347A344434403413
:1034D0001C3446345034C3344734243474344934AF
:1034E000973418344B34BC34BE344C346B346E34A3
:1034F0004E340334153450347934AD346034F334FD
:1035000049347134AE34C834A134A634B0348D3467
:10351000143420340234AF34013400340034003425
:103520000A3400340034003464340034003400348D
:10353000E8340334003400341034273400340034C9
:10354000A034863401340034403442340F34003423
:1035500080349634983400340034E134F534053442
:103560000034CA349A343B34443426340B34143493
:103570009134603445341F3400341B341B3485349B
:1035800000340034003452346534633465347034AC
:1035900074346534753472342034413453344B34CC
:1035A0002034563431342E343034003446347234BE
:1035B00065347134203476346134723420342D34DF
:1035C0002F342B34313430344D3448347A34003491
:1035D00046347234653471343D34253437342E34F6
:1035E0003334663420344D3468347A340034523401
:1035F0005334533449343D34253433346434203423
:0A36000020342534333464340034E0
:020000040001F9
:04000E0084CFFBD7C9
:00000001FF
